:1000000083168601EF308500C13081008312A5017F
:10001000A701A901A801C830AB00F630AE00A120AD
:10002000051D1B280130AC001430A9002814A814A9
:100030004B20F6203D28AC014B208730FC2064008B
:100040001F288207C034F934A434B0349934923470
:100050008234F8348034903482073134B734313408
:10006000743431347E34313488343134943431341E
:10007000AB3430342A3431345634A120E620AA0B74
:100080003D2864001130AA00BF20AB0B3D2828306A
:10009000AB00A7203D2803102C0DA6002C20A100AA
:1000A000260A2C20A0006430A4000310A00DA10D8E
:1000B00020146620C4307320200873202108732088
:1000C00024087320003073208E2008000C30831623
:1000D00085008312851400000514000085100000BF
:1000E000051000000800A3000C3083168500831261
:1000F0000830A200A30D8514031C85100000051410
:10010000000005100000A20B7A280E30831685002F
:100110008312051400000510000008000C3083163F
:10012000850083128510000005140000851400006E
:100130000F308316850083120800FE30AE00AD013B
:1001400008000B1DA128B93081000B110800A90877
:100150000319B4288519BD284B30A900A81CB32861
:10016000D230AE00A8100800281CB928F0204B207F
:10017000F620A8141430A900B328A903B328A708AF
:10018000031DCE280519CD289D20A5010A30A70002
:100190002818E028F0204B20F62008000519DE285A
:1001A0000A30A700A50A64302502031DCD282814B3
:1001B000A8141430A90086139D20CD28A703CD28AC
:1001C0000F30A900A81028108617CD28AE080319F3
:1001D000EF280130AD070318AE0A1030850608007D
:1001E00007302C020318AC01AC0A08002C082120AF
:0C01F000FC202818861308008600080078
:02400E00FD3F74
:00000001FF
